:020000040000FA
:1000000083169B0108308100003085000730860090
:10001000831285010230A400061D232828203620E3
:1000200005102408A3005A2000000130A302031D7C
:10003000132805142408A3005A2000000130A3024D
:10004000031D1C280C2805105A2005145A200C28C2
:10005000061835281430A4074C20E6302402031972
:100060003528031C3528E630A400080086184428EB
:100070001430A4024C200000E63024020319442866
:10008000031C44280230A40008004230A000A00B4A
:100090004728000000000800BA30A0000430A1008A
:1000A0000230A200A00B5228A10B5228A20B52280A
:1000B000000008002130A000A00B5C280000000018
:0200C000080036
:02400E002A3F47
:02401000FC3F73
:00000001FF
